:100000000C942A000C943C000C943C000C943C0092
:100010000C943C000C943C000C943C000C943C0070
:100020000C943C000C943C000C943C000C94790023
:100030000C943C000C943C000C943C000C943C0050
:100040000C943C000C943C000C943C000C943C0040
:100050000C943C0011241FBECFE5D4E0DEBFCDBF21
:1000600010E0A0E6B0E001C01D92A23AB107E1F7AE
:100070000E943E000C9437010C9400001F93CF9314
:10008000DF9380EA91E00E946A008FEF85BBC0E0B9
:10009000D0E013B38AE40E94FE0081E40E94FE00D7
:1000A00081E40E94FE00812F0E94FE00812F809536
:1000B0000E94FE008AE50E94FE00CE010197F1F742
:1000C000CE010197F1F7CE010197F1F7CE0101972B
:1000D000F1F7DFCF2FEF2093610020916100209393
:1000E000600090BD89B986E880BD88E88AB97894B7
:1000F00008951F920F920FB60F9211242F933F93E2
:100100004F938F939F93EF93FF934CB18091610036
:100110008F3389F18091610020916000992787FDDC
:1001200090950196332727FD30958217930739F173
:10013000809161008F3391F1809161008F5F809396
:100140006100E0916100FF27E7FDF095EE59FF4F58
:100150004083809160008F3F11F410926000FF9106
:10016000EF919F918F914F913F912F910F900FBEE3
:100170000F901F90189580916000882359F6809108
:1001800060008F5F8093600080916000803481F612
:1001900010926000809161008F3371F610926100BF
:1001A000D0CF809160008F3FC9F0E0916000FF27C1
:1001B000E7FDF095EE59FF4FE0819091600080914E
:1001C0006100981771F0809160008F5F80936000EC
:1001D00080916000803471F08E2F0895E0E08E2FC2
:1001E00008958FEF8093610080916100809360009B
:1001F0008E2F0895109260008E2F08955D9BFECF84
:100200008CB90895809160008F3FE1F0909160007B
:1002100080916100981774F0909160008091610066
:1002200089179CF490916100809160009F5B981BFE
:10023000892F089590916100809160009F5F981BC5
:10024000892F089590E0892F089591E0892F0895CE
:10025000FC018081882339F05D9BFECF8CB93196FB
:1002600080818823C9F75D9BFECF1CB80895F89460
:02027000FFCFBE
:00000001FF
